Microchip MPLAB XC8 Compiler V2.36

Linker command line:

-W-3 --edf=/opt/microchip/xc8/v2.36/pic/dat/en_msgs.txt -cn \
  -h+dist/default/production/PRUEBA_FUNCIONA.X.production.sym \
  --cmf=dist/default/production/PRUEBA_FUNCIONA.X.production.cmf -z \
  -Q18F452 -o/tmp/xcXNeBFMd --defsym=__MPLAB_BUILD=1 \
  -Mdist/default/production/PRUEBA_FUNCIONA.X.production.map \
  --md=/tmp/xcXJJcnfj.dat -E1 -ver=XC8 Compiler --acfsm=1493 \
  -ACODE=00h-03FFFhx2 -ACONST=00h-07FFFh -ASMALLCONST=0600h-06FFhx122 \
  -AMEDIUMCONST=0600h-07FFFh -ACOMRAM=01h-07Fh -AABS1=00h-05FFh \
  -ABIGRAM=01h-05FFh -ARAM=080h-0FFh,0100h-01FFhx5 -ABANK0=080h-0FFh \
  -ABANK1=0100h-01FFh -ABANK2=0200h-02FFh -ABANK3=0300h-03FFh \
  -ABANK4=0400h-04FFh -ABANK5=0500h-05FFh -ASFR=0F80h-0FFFh \
  -ABIGSFR=0F80h-0FFFh -ACONFIG=0300000h-030000Dh -AIDLOC=0200000h-0200007h \
  -AEEDATA=0F00000h-0F000FFh -peeprom_data=EEDATA \
  -preset_vec=00h,intcode,intcodelo,powerup,init -pramtop=0600h \
  -psmallconst=SMALLCONST -pmediumconst=MEDIUMCONST -pconst=CONST \
  -AFARRAM=00h-00h \
  -prdata=COMRAM,nvrram=COMRAM,nvbit=COMRAM,rbss=COMRAM,rbit=COMRAM \
  -pfarbss=FARRAM,fardata=FARRAM,nvFARRAM=FARRAM \
  -pintsave_regs=BIGRAM,bigbss=BIGRAM,bigdata=BIGRAM -pbss=RAM \
  -pidata=CODE,irdata=CODE,ibigdata=CODE,ifardata=CODE -prparam=COMRAM \
  /tmp/xcXlGJmcB.o dist/default/production/PRUEBA_FUNCIONA.X.production.o 

Object code version is 3.11

Machine type is 18F452



                Name                               Link     Load   Length Selector   Space Scale
/tmp/xcXlGJmcB.o
                idloc                            200000   200000        8        0       5
                config                           300000   300000        E        0       4
                text                               2D4A     2D4A        2     16A5       0
                init                                  2        2        4        0       0
                reset_vec                             0        0        2        0       0
dist/default/production/PRUEBA_FUNCIONA.X.production.o
                idloc                            200000   200000        8        0       5
                config                           300000   300000        E        0       4
                text5                              3A56     3A56      5AA     1D2B       0
                text4                              3180     3180      432     18C0       0
                text3                              35B2     35B2      4A4     1AD9       0
                text2                              2E04     2E04      136     1702       0
                text1                              2F3A     2F3A      246     179D       0
                text0                              2D7C     2D7C       88     16BE       0
                cstackCOMRAM                          1        1       6E        1       1
                dataCOMRAM                           7B       7B        3        1       1
                bssCOMRAM                            7E       7E        2        1       1
                cinit                              2D50     2D50       2C     16A8       0
                nvCOMRAM                             6F       6F        C        1       1
                idataCOMRAM                        2D4D     2D4D        3     2D4D       0

TOTAL           Name                               Link     Load   Length     Space
        CLASS   CODE           
                text                               2D4A     2D4A        2         0
                init                                  2        2        4         0
                reset_vec                             0        0        2         0
                text5                              3A56     3A56      5AA         0
                text4                              3180     3180      432         0
                text3                              35B2     35B2      4A4         0
                text2                              2E04     2E04      136         0
                text1                              2F3A     2F3A      246         0
                text0                              2D7C     2D7C       88         0
                cinit                              2D50     2D50       2C         0
                idataCOMRAM                        2D4D     2D4D        3         0

        CLASS   CONST          

        CLASS   SMALLCONST     

        CLASS   MEDIUMCONST    

        CLASS   COMRAM         
                cstackCOMRAM                          1        1       6E         1
                dataCOMRAM                           7B       7B        3         1
                bssCOMRAM                            7E       7E        2         1
                nvCOMRAM                             6F       6F        C         1

        CLASS   ABS1           

        CLASS   BIGRAM         

        CLASS   RAM            

        CLASS   BANK0          

        CLASS   BANK1          

        CLASS   BANK2          

        CLASS   BANK3          

        CLASS   BANK4          

        CLASS   BANK5          

        CLASS   SFR            

        CLASS   BIGSFR         

        CLASS   CONFIG         
                config                           300000   300000        E         4

        CLASS   IDLOC          
                idloc                            200000   200000        8         5

        CLASS   EEDATA         

        CLASS   FARRAM         

        CLASS   HEAP           

        CLASS   STACK          



SEGMENTS        Name                           Load    Length   Top    Selector   Space  Class

                text1                          002F3A  000246  003180      179D       0  CODE    
                text2                          002E04  000136  002F3A      1702       0  CODE    
                reset_vec                      000000  000006  000006         0       0  CODE    
                text4                          003180  000432  0035B2      18C0       0  CODE    
                text0                          002D7C  000088  002E04      16BE       0  CODE    
                text3                          0035B2  0004A4  003A56      1AD9       0  CODE    
                text5                          003A56  0005AA  004000      1D2B       0  CODE    
                cinit                          002D50  00002C  002D7C      16A8       0  CODE    
                text                           002D4A  000002  002D4C      16A5       0  CODE    
                idataCOMRAM                    002D4D  000003  002D50      2D4D       0  CODE    
                cstackCOMRAM                   000001  00007F  000080         1       1  COMRAM  


UNUSED ADDRESS RANGES

        Name                Unused          Largest block    Delta
        BANK0            000080-0000FF               80
        BANK1            000100-0001FF              100
        BANK2            000200-0002FF              100
        BANK3            000300-0003FF              100
        BANK4            000400-0004FF              100
        BANK5            000500-0005FF              100
        BIGRAM           000080-0005FF              580
        BIGSFR           000F80-000FFF               80
        CODE             000006-002D49             2D44
                         002D4C-002D4C                1
                         004000-007FFF             4000
        CONST            000006-002D49             2D44
                         002D4C-002D4C                1
                         004000-007FFF             4000
        EEDATA           F00000-F000FF              100
        MEDIUMCONST      000600-002D49             274A
                         002D4C-002D4C                1
                         004000-007FFF             4000
        RAM              000080-0005FF              100
        SFR              000F80-000FFF               80
        SMALLCONST       000600-002D49              100
                         002D4C-002D4C                1
                         004000-007FFF              100

                                  Symbol Table

?___fladd                                                             cstackCOMRAM 000033
?___fldiv                                                             cstackCOMRAM 000001
?___flmul                                                             cstackCOMRAM 00001A
?___fltol                                                             cstackCOMRAM 000043
_ACKDT                                                                (abs)        007E2D
_ACKEN                                                                (abs)        007E2C
_ACKSTAT                                                              (abs)        007E2E
_BackLight_State                                                      dataCOMRAM   00007D
_CCP1CON                                                              (abs)        000FBD
_CCPR1L                                                               (abs)        000FBE
_LATBbits                                                             (abs)        000F8A
_PEN                                                                  (abs)        007E2A
_PR2                                                                  (abs)        000FCB
_RCEN                                                                 (abs)        007E2B
_RS                                                                   bssCOMRAM    00007F
_RSEN                                                                 (abs)        007E29
_SEN                                                                  (abs)        007E28
_SSPADD                                                               (abs)        000FC8
_SSPBUF                                                               (abs)        000FC9
_SSPCON1                                                              (abs)        000FC6
_SSPCON2                                                              (abs)        000FC5
_SSPIF                                                                (abs)        007CF3
_SSPSTAT                                                              (abs)        000FC7
_T2CON                                                                (abs)        000FCA
_TRISBbits                                                            (abs)        000F93
_TRISC3                                                               (abs)        007CA3
_TRISC4                                                               (abs)        007CA4
_TRISCbits                                                            (abs)        000F94
__HRAM                                                                (abs)        000000
__Habs1                                                               abs1         000000
__Hbank0                                                              bank0        000000
__Hbank1                                                              bank1        000000
__Hbank2                                                              bank2        000000
__Hbank3                                                              bank3        000000
__Hbank4                                                              bank4        000000
__Hbank5                                                              bank5        000000
__Hbigbss                                                             bigbss       000000
__Hbigdata                                                            bigdata      000000
__Hbigram                                                             bigram       000000
__Hbigsfr                                                             bigsfr       000000
__Hbss                                                                bss          000000
__HbssCOMRAM                                                          bssCOMRAM    000000
__Hcinit                                                              cinit        000000
__Hclrtext                                                            clrtext      000000
__Hcomram                                                             comram       000000
__Hconfig                                                             config       30000E
__Hconst                                                              const        000000
__HcstackCOMRAM                                                       cstackCOMRAM 000000
__Hdata                                                               data         000000
__HdataCOMRAM                                                         dataCOMRAM   000000
__Heeprom_data                                                        eeprom_data  000000
__Hfarbss                                                             farbss       000000
__Hfardata                                                            fardata      000000
__Hheap                                                               heap         000000
__Hibigdata                                                           ibigdata     000000
__Hidata                                                              idata        000000
__HidataCOMRAM                                                        idataCOMRAM  000000
__Hidloc                                                              idloc        200008
__Hifardata                                                           ifardata     000000
__Hinit                                                               init         000006
__Hintcode                                                            intcode      000002
__Hintcode_body                                                       intcode_body 000000
__Hintcodelo                                                          intcodelo    000002
__Hintentry                                                           intentry     000000
__Hintret                                                             intret       000000
__Hintsave_regs                                                       intsave_regs 000000
__Hirdata                                                             irdata       000000
__Hmediumconst                                                        mediumconst  000000
__HnvCOMRAM                                                           nvCOMRAM     000000
__HnvFARRAM                                                           nvFARRAM     000000
__Hnvbit                                                              nvbit        000000
__Hnvrram                                                             nvrram       000000
__Hparam                                                              rparam       000000
__Hpowerup                                                            powerup      000002
__Hram                                                                ram          000000
__Hramtop                                                             ramtop       000600
__Hrbit                                                               rbit         000000
__Hrbss                                                               rbss         000000
__Hrdata                                                              rdata        000000
__Hreset_vec                                                          reset_vec    000002
__Hrparam                                                             rparam       000000
__Hsfr                                                                sfr          000000
__Hsmallconst                                                         smallconst   000000
__Hspace_0                                                            (abs)        004000
__Hspace_1                                                            (abs)        000080
__Hspace_2                                                            (abs)        000000
__Hspace_4                                                            (abs)        60000E
__Hstack                                                              stack        000000
__Hstruct                                                             struct       000000
__Htemp                                                               temp         000000
__Htext                                                               text         000000
__Htext0                                                              text0        000000
__Htext1                                                              text1        000000
__Htext2                                                              text2        000000
__Htext3                                                              text3        000000
__Htext4                                                              text4        000000
__Htext5                                                              text5        000000
__LRAM                                                                (abs)        000001
__Labs1                                                               abs1         000000
__Lbank0                                                              bank0        000000
__Lbank1                                                              bank1        000000
__Lbank2                                                              bank2        000000
__Lbank3                                                              bank3        000000
__Lbank4                                                              bank4        000000
__Lbank5                                                              bank5        000000
__Lbigbss                                                             bigbss       000000
__Lbigdata                                                            bigdata      000000
__Lbigram                                                             bigram       000000
__Lbigsfr                                                             bigsfr       000000
__Lbss                                                                bss          000000
__LbssCOMRAM                                                          bssCOMRAM    000000
__Lcinit                                                              cinit        000000
__Lclrtext                                                            clrtext      000000
__Lcomram                                                             comram       000000
__Lconfig                                                             config       000000
__Lconst                                                              const        000000
__LcstackCOMRAM                                                       cstackCOMRAM 000000
__Ldata                                                               data         000000
__LdataCOMRAM                                                         dataCOMRAM   000000
__Leeprom_data                                                        eeprom_data  000000
__Lfarbss                                                             farbss       000000
__Lfardata                                                            fardata      000000
__Lheap                                                               heap         000000
__Libigdata                                                           ibigdata     000000
__Lidata                                                              idata        000000
__LidataCOMRAM                                                        idataCOMRAM  000000
__Lidloc                                                              idloc        000000
__Lifardata                                                           ifardata     000000
__Linit                                                               init         000002
__Lintcode                                                            intcode      000002
__Lintcode_body                                                       intcode_body 000000
__Lintcodelo                                                          intcodelo    000002
__Lintentry                                                           intentry     000000
__Lintret                                                             intret       000000
__Lintsave_regs                                                       intsave_regs 000000
__Lirdata                                                             irdata       000000
__Lmediumconst                                                        mediumconst  000000
__LnvCOMRAM                                                           nvCOMRAM     000000
__LnvFARRAM                                                           nvFARRAM     000000
__Lnvbit                                                              nvbit        000000
__Lnvrram                                                             nvrram       000000
__Lparam                                                              rparam       000000
__Lpowerup                                                            powerup      000002
__Lram                                                                ram          000000
__Lramtop                                                             ramtop       000600
__Lrbit                                                               rbit         000000
__Lrbss                                                               rbss         000000
__Lrdata                                                              rdata        000000
__Lreset_vec                                                          reset_vec    000000
__Lrparam                                                             rparam       000000
__Lsfr                                                                sfr          000000
__Lsmallconst                                                         smallconst   000000
__Lspace_0                                                            (abs)        000000
__Lspace_1                                                            (abs)        000000
__Lspace_2                                                            (abs)        000000
__Lspace_4                                                            (abs)        000000
__Lstack                                                              stack        000000
__Lstruct                                                             struct       000000
__Ltemp                                                               temp         000000
__Ltext                                                               text         000000
__Ltext0                                                              text0        000000
__Ltext1                                                              text1        000000
__Ltext2                                                              text2        000000
__Ltext3                                                              text3        000000
__Ltext4                                                              text4        000000
__Ltext5                                                              text5        000000
__S0                                                                  (abs)        004000
__S1                                                                  (abs)        000080
__S4                                                                  (abs)        000000
__S5                                                                  (abs)        000000
___fladd                                                              text5        003A56
___fladd@a                                                            cstackCOMRAM 000037
___fladd@aexp                                                         cstackCOMRAM 000040
___fladd@b                                                            cstackCOMRAM 000033
___fladd@bexp                                                         cstackCOMRAM 000041
___fladd@grs                                                          cstackCOMRAM 000042
___fladd@signs                                                        cstackCOMRAM 00003F
___fldiv                                                              text4        003180
___fldiv@a                                                            cstackCOMRAM 000005
___fldiv@aexp                                                         cstackCOMRAM 000019
___fldiv@b                                                            cstackCOMRAM 000001
___fldiv@bexp                                                         cstackCOMRAM 000018
___fldiv@grs                                                          cstackCOMRAM 000014
___fldiv@new_exp                                                      cstackCOMRAM 000012
___fldiv@rem                                                          cstackCOMRAM 00000D
___fldiv@sign                                                         cstackCOMRAM 000011
___flmul                                                              text3        0035B2
___flmul@a                                                            cstackCOMRAM 00001E
___flmul@aexp                                                         cstackCOMRAM 00002B
___flmul@b                                                            cstackCOMRAM 00001A
___flmul@bexp                                                         cstackCOMRAM 00002C
___flmul@grs                                                          cstackCOMRAM 000027
___flmul@prod                                                         cstackCOMRAM 00002D
___flmul@sign                                                         cstackCOMRAM 000026
___flmul@temp                                                         cstackCOMRAM 000031
___fltol                                                              text2        002E04
___fltol@exp1                                                         cstackCOMRAM 00004C
___fltol@f1                                                           cstackCOMRAM 000043
___fltol@sign1                                                        cstackCOMRAM 00004B
___heap_hi                                                            (abs)        000000
___heap_lo                                                            (abs)        000000
___inthi_sp                                                           stack        000000
___intlo_sp                                                           stack        000000
___param_bank                                                         (abs)        000000
___rparam_used                                                        (abs)        000001
___sp                                                                 stack        000000
__accesstop                                                           (abs)        000080
__activetblptr                                                        (abs)        000002
__cntErrataNOP_/tmp/xcXlGJmcB.o                                       (abs)        000001
__cntErrataNOP_dist/default/production/PRUEBA_FUNCIONA.X.production.o (abs)        00010E
__end_of___fladd                                                      text5        003FFE
__end_of___fldiv                                                      text4        0035B2
__end_of___flmul                                                      text3        003A56
__end_of___fltol                                                      text2        002F3A
__end_of__initialization                                              cinit        002D72
__end_of_main                                                         text0        002E04
__end_of_setPWM                                                       text1        003180
__initialization                                                      cinit        002D50
__mediumconst                                                         mediumconst  000000
__pbssCOMRAM                                                          bssCOMRAM    00007E
__pcinit                                                              cinit        002D50
__pcstackCOMRAM                                                       cstackCOMRAM 000001
__pdataCOMRAM                                                         dataCOMRAM   00007B
__pidataCOMRAM                                                        idataCOMRAM  002D4D
__pnvCOMRAM                                                           nvCOMRAM     00006F
__ptext0                                                              text0        002D7C
__ptext1                                                              text1        002F3A
__ptext2                                                              text2        002E04
__ptext3                                                              text3        0035B2
__ptext4                                                              text4        003180
__ptext5                                                              text5        003A56
__ramtop                                                              ramtop       000600
__smallconst                                                          smallconst   000000
_frec_osc                                                             nvCOMRAM     000073
_i2c_add                                                              bssCOMRAM    00007E
_main                                                                 text0        002D7C
_mask                                                                 dataCOMRAM   00007B
_pwm_p                                                                nvCOMRAM     000077
_setPWM                                                               text1        002F3A
_setPWM$946                                                           cstackCOMRAM 000069
_setPWM$947                                                           cstackCOMRAM 000061
_tmr2_presc                                                           nvCOMRAM     00006F
end_of_initialization                                                 cinit        002D72
intlevel0                                                             text         002D4A
intlevel1                                                             text         002D4A
intlevel2                                                             text         002D4A
intlevel3                                                             text         002D4A
isa$std                                                               (abs)        000001
isa$xinst                                                             (abs)        000000
setPWM@duty_temp                                                      cstackCOMRAM 000067
setPWM@freq_osc                                                       cstackCOMRAM 000055
setPWM@period_pwm                                                     cstackCOMRAM 00004D
setPWM@periodo                                                        cstackCOMRAM 000065
setPWM@presc                                                          cstackCOMRAM 000059
setPWM@pwm_duty                                                       cstackCOMRAM 000051
setPWM@valor_prueba_debug                                             cstackCOMRAM 00005F
setPWM@valor_prueba_debug2                                            cstackCOMRAM 000060
stackhi                                                               (abs)        000000
stacklo                                                               (abs)        000000
start                                                                 init         000002
start_initialization                                                  cinit        002D50


MODULE INFORMATION

Module		Function		Class		Link	Load	Size
/opt/microchip/xc8/v2.36/pic/sources/c99/common/sprcmul.c
		___flmul       		CODE           	35B2	0000	1188

/opt/microchip/xc8/v2.36/pic/sources/c99/common/sprcmul.c estimated size: 1188

/opt/microchip/xc8/v2.36/pic/sources/c99/common/sprcdiv.c
		___fldiv       		CODE           	3180	0000	1074

/opt/microchip/xc8/v2.36/pic/sources/c99/common/sprcdiv.c estimated size: 1074

shared
		__initialization		CODE           	2D50	0000	34

shared estimated size: 34

/opt/microchip/xc8/v2.36/pic/sources/c99/common/fltol.c
		___fltol       		CODE           	2E04	0000	310

/opt/microchip/xc8/v2.36/pic/sources/c99/common/fltol.c estimated size: 310

/opt/microchip/xc8/v2.36/pic/sources/c99/common/sprcadd.c
		___fladd       		CODE           	3A56	0000	1448

/opt/microchip/xc8/v2.36/pic/sources/c99/common/sprcadd.c estimated size: 1448

main.c
		_main          		CODE           	2D7C	0000	136
		_setPWM        		CODE           	2F3A	0000	582

main.c estimated size: 718

